:1000000000308A00122A0000FF00030E8301A100C5
:100010007F08A0000A08A8008A01A00E0408A20018
:100020007708A3007808A4007908A5007A08A6003C
:100030007B08A700831383128C308400001C2228C5
:100040000C183B288C308400801C28288C183D28F4
:10005000220884002308F7002408F8002508F90086
:100060002608FA002708FB0028088A00210E8300D2
:10007000FF0E7F0E09008A113F288A115328301481
:100080000C108A1128280830C002031C5228403066
:1000900084000310800C00080319522850286400C3
:1000A000800B4F2800348316861283128616640054
:1000B0000930BF006D30C0004320BF0B5A282C0808
:1000C000BE00BE0803196A2864000000000000009A
:1000D000BE03612883168612831286128C108A1141
:1000E00028283D3084000008031988280230F800D1
:1000F000BF30F7006400F70B7A28F80B78289630A9
:10010000F700F70B8128000000006400800B7628C0
:100110000034B90183160513831205138316851362
:100120008312851783160510831205108316851018
:10013000831285140230BC00C830BD007120BC0B96
:100140009C288316051383120513831685138312C7
:1001500085138316051083120510831685108312EC
:100160008510E130AC006430BD00712083160510AD
:100170008312051083168510831285148316851348
:10018000831285138316051383120517C830BD002B
:100190007120AA1FDA281308930183161418D22895
:1001A0008312CD2883121308AA00AA090430BD00C7
:1001B0007120C92883160510831205108316851037
:1001C0008312851083160513831205138316851376
:1001D00083128513BB01BA013B08033C031C57295A
:1001E000031DF6283A08E73C031C5729831685159A
:1001F0008312851926290108B43C031C082983169B
:10020000051083120510831685108312851410299A
:10021000831605108312051083168510831285102E
:100220000108A03C031C1D29831685138312851326
:1002300083160513831205172529831605138312C8
:100240000513831685138312851350290108B43CC6
:10025000031C33298316851083128510831605101D
:10026000831205143B29831605108312051083168B
:100270008510831285100108A03C031C48298316B1
:1002800005138312051383168513831285175029CE
:1002900083160513831205138316851383128513A2
:1002A0000130BD007120BA0A0319BB0AEC2883167D
:1002B0000513831205138316851383128513831682
:1002C0000510831205108316851083128510803067
:1002D000AC006430BD007120831685138312851332
:1002E0008316051383120517831685108312851054
:1002F00083160510831205140230BC00FA30BD00CD
:100300007120BC0B7E2983160510831205108316FD
:100310008510831285148316051383120513831623
:10032000851383128517C830BD0071208316051010
:10033000831205108316851083128510831605130A
:10034000831205138316851383128513AD30AC0019
:100350006430BD00712083168510831285108316CA
:100360000510831205140230BC00C830BD00712096
:10037000BC0BB5299930AC0083168510831285100B
:1003800083160510831205148316851383128513B3
:1003900083160513831205176430BD0071208A305F
:1003A000AC00831685108312851083160510831206
:1003B0000514831685138312851383160513831280
:1003C0000517C830BD0071202A087F390319F729A5
:1003D0001308930183161418EF298312EA29831254
:1003E0001308AA00AA090430BD007120E42983166D
:1003F0000510831205108316851083128514831649
:100400000513831205138316851383128517023093
:10041000BC00C830BD007120BC0B092A5330AC00B1
:100420008A11432B84011F308305703083168F009F
:100430001F129F121B0880399B0007309C008312FB
:10044000AB0183161F129F121B08803974389B0062
:100450001F1383121F179F1783169F1383121F14D6
:1004600094128316061186140612313083129400FA
:100470000030831694000108C739083881003030F5
:10048000831290007830F800063892008C30831682
:10049000920072308F0005138312051383168513A3
:1004A0008312851383160510831205108316851099
:1004B00083128510B201B101B401B3018030AC00E8
:1004C000AF0183168C14C03083128B04831606117F
:1004D000831206110630B900FA30BD007120B90B45
:1004E0006C2A2830F8001F08C73978049F000130B3
:1004F000BD0071201F151F197B2A1E08F700F70C7D
:10050000F70C3F30F7057708643EAD003030F80057
:100510001F08C73978049F000130BD0071202030CA
:100520002D02B9001F151F19932A1E08F700F70C9A
:10053000F70C3F30F70577083907AE000108801F38
:10054000A42AB21FAC2AA62AB21BB52AB208031DE0
:10055000AC2A3102031CB52A83168510831285103C
:100560008316051083120514BD2A83160510831205
:10057000051083168510831285100108801FC32A79
:10058000B41FCB2AC52AB41BD42AB408031DCB2A16
:100590003302031CD42A8316851383128513831612
:1005A000051383120517DC2A83160513831205131E
:1005B000831685138312851364000130BD007120FA
:1005C0000930B900A9018B1BA9178B136D30C0002E
:1005D0004320A91B8B17B90BE22A8316061083123E
:1005E00006101308930183161418F82A8312F32AAD
:1005F00083121308AA00AA09831606108312061490
:10060000B601B5013508063C031C142B2A08F70077
:100610003508F8000319102B0310F70CF80B0C2BFE
:100620007718B60AB50A022B3608033C0318402B8C
:100630008316051083120510831685108312851406
:1006400083160513831205138316851383128517EA
:100650000230B9009630BD007120B90B2A2B8316E9
:1006600005138312051383168513831285138316CE
:1006700005108312051083168510831285103F2BF9
:10068000AA1F432B8928AA1D612B8030AC002F089C
:10069000313C031C512BB201FF30B100B401B30057
:1006A0005B2BFA012D08B1007A08B200FA012D087F
:1006B000B3007A08B400AB012F0F5F2B602BAF0A99
:1006C0009E2A2A1C6F2B5330AC00B201B101FA01F3
:1006D0002E08B3007A08B4000330AB009E2A2A1F0C
:1006E0007D2BAD30AC00B401B301FA012E08B1008E
:1006F0007A08B200FD30AB009E2AAA1C8F2B67300F
:10070000AC0032302D02FA01B1007A08B200FA01D1
:100710002D08B3007A08B4000230AB009E2AAA1E4E
:10072000A12B9930AC0032302D02FA01B3007A08C7
:10073000B400FA012D08B1007A08B200FE30AB0017
:100740009E2A2A1DB62B7630AC00FA012D08B10086
:100750007A08B200FA012D08B3007A08B40001301B
:10076000AB002F0FB42BB52BAF0A9E2A2A1ECB2B22
:100770008A30AC00FA012D08B3007A08B400FA01FF
:100780002D08B1007A08B200FF30AB002F0FC92B43
:10079000CA2BAF0A9E2A2B08033C0319D32B2B0824
:1007A000FD3C031DF22B2F08323C0318F12B83165E
:1007B0000510831205108316851083128514831685
:1007C000051383120513831685138312851764306E
:1007D000BD0071202F08FA3C0318F12B3230BD0008
:0807E0007120AF019E2A6300A5
:04400E00383FFC3FFC
:00000001FF
